:020000040000FA
:040000000000F328E1
:080008008C1061080319132894
:10001000E11C0E280518E028E1100900051CCE2877
:10002000D001D101E10162182428050806396502D2
:10003000031D1E28E70B8A28E2148A286214033065
:10004000E3000F30E7008A28E30B8A28050C033908
:10005000E600650D0C3966070F39DF0000308A00B5
:100060005F08820742286C284728422847284228F0
:1000700042286C286C2842284228472842284728D2
:100080006C284228621005080639E5008A28050810
:100090000639E500E21C4E2801304F280830E20105
:1000A000D007031C55280130D10758085002D4004E
:1000B000031C602859085102D500031867288A28B4
:1000C000013059075102D500031867288A285408BF
:1000D000D0005508D1008A2805080639E500E21C41
:1000E0007328013074280830E201D00203188A28EE
:1000F0000130D10203188A285908D1075808D007BF
:10010000031C84280130D1070130D007031C8A2842
:10011000D1078A28601050085202D400031C962888
:1001200051085302D500031C9C28A5280130510713
:100130005302D5000318A5286014D509D40901304D
:10014000D407031CA5280130D507D408031DAB280C
:10015000D5080319090054085602031CB428550891
:100160005702031CBA28BC28013055075702031C4C
:10017000BA28BC280130E006601CD028D008031D36
:10018000C928D108031DC9285808D0005908D10032
:10019000CE280130D0020318CE28D102E403E12892
:1001A00058085002031DDB2859085102031DDB28A3
:1001B000D001D101E0280130D007031CE028D1078D
:1001C000E40A64080739E62086000900DF000030F1
:1001D0008A005F0882079034103450344034603411
:1001E0002034A0348034D001D101D201D3011F309A
:1001F000D8000330D9009030D6000130D70003304A
:10020000E1004130C000BD01C101C201C301C40110
:10021000C501C601C701C801DC012030B800831246
:10022000B901380884003908840783169B001C1420
:100230001A0883128000B90A0F303902031D1129F0
:100240005A30B200B300B4003930B500B6003230D5
:10025000B000B1012930B800B901BA01BB01BD013C
:1002600007309F0083160F308600FF308500831211
:100270008316BE30920083120F30920083164D30E9
:100280009900203098008312903098008B170B173C
:1002900083168C1483128B178C1A5129DC1B2D2A80
:1002A0004C298B131A08BC008C123B18AA29BA1BC4
:1002B0008029300884003108840700083C02031DAF
:1002C0006B29B10A05303102031D6C29B101B90156
:1002D000FF30BA004B29B10138088400390884077F
:1002E00000083C02031D7E29B90A05303902031DAE
:1002F0004B29B101B901FF30BA004B29B9014B2993
:100300003C08BA00FF30BB0001308A003A080F39C0
:100310009521CD004D080319B829BD01DE01CD1F7F
:100320004B29CD132808DE004B29DF0001308A005D
:100330005F08820700340234823400340034003411
:100340000034003400340534013400340034003407
:1003500000340034DE080319AF29DE034B294008BE
:1003600084003D0884073C088000BD0ACD0B4B2962
:10037000BD01BB0101308A003A080F39C23E0318A3
:100380008A0A8200F328D229D229F328F328F328F5
:10039000F328F328ED29FF29F529F328F328F3287A
:1003A000F328F32841085802031CDF2942085902A8
:1003B000031CE8294108D2004208D3004B29420817
:1003C0005902031CE829DF0001305F020318DA2913
:1003D0005808D2005908D3004B290830DB001130EF
:1003E000DD008130DC00BA014B294108A80008304B
:1003F000DB002830DA000130BE00BA01102A4108C3
:10040000A9004208AA004308AB004408AC00450814
:10041000AD000930DB002930DA000530BE00BA013A
:100420005A088400000883169A0083125B0883161A
:100430009B009C111C1555309D00AA309D009C14FA
:100440001C1183128C1F222A8C13DB0ADA0ABE0BC2
:10045000102AB901BA01BB014B298B130C1E4B2981
:100460005B0883169B001C141A0883129900DB0A90
:08047000DD0B4B29DC014B29D7
:02400E00613F10
:1042000000000000000000000000000000000000AE
:10421000000044004700300030003100200053000F
:104220005400500052002000560031002E00300093
:04423000300030002A
:00000001FF
